:1000000003F901210001051401060105140106018F
:100010000514010601051401060105140106010578
:100020001401060105140106010514010601051459
:10003000010601051401060105140106010514015C
:100040000601051401060105140106010514010647
:10005000010514010601051401060105140106013C
:100060000514010601051401060105140106010528
:100070001401060105140106010514010601051409
:10008000010601051401060105140106010514010C
:1000900006010514010601051401060105140106F7
:1000A00001051401060105140106010514010601EC
:1000B00005140106010514010601051401060105D8
:1000C00014010601051401060105140106010514B9
:1000D00001060105140106010514010601051401BC
:1000E00006010514010601051401060105140106A7
:1000F000010514010601051401060105140106019C
:100100000514010601051401060105140106010587
:100110001401060105140106010514010601051468
:10012000010601051401060105140106010514016B
:100130000601051401060105140106010514010656
:10014000010514010601051401060105140106014B
:100150000514010601051401060105140106010537
:100160001401060105140106010514010601051418
:10017000010601051401060105140106010514011B
:100180000601051401060105140106010514010606
:1001900001051401060105140106010514010601FB
:1001A00005140106010514010601051401060105E7
:1001B00014010601051401060105140106010514C8
:1001C00001060105140106010514010601051401CB
:1001D00006010514010601051401060105140106B6
:1001E00001051401060105140106010514010601AB
:1001F000051401060105140106010514010622007B
:00000001FF
